:020000040800F2
:10000000580D0020C500000899180008F5160008D2
:1000100000000000000000000000000000000000E0
:10002000000000000000000000000000BD180008F3
:1000300000000000000000009B180008611A000882
:10004000D700000800000000D7000008D700000813
:10005000D7000008D7000008D7000008690800088A
:1000600000000000D7000008D7000008D7000008F3
:10007000D7000008D7000008D700000800000000E3
:10008000D70000080000000000000000D7000008B2
:1000900000000000D7000008D7000008D7000008C3
:1000A00000000000D700000800000000D700000892
:1000B0000348854600F028FB00480047D92B00087C
:1000C000580D00200448804704480047FEE7FEE73B
:1000D000FEE7FEE7FEE7FEE7CB1A0008B1000008E6
:1000E00030B50B46014600202022012409E00D46D0
:1000F000D5409D4205D31D469540491B2546954058
:1001000040191546521E002DF1DC30BD70B500249B
:100110002546002801DA01244042002901DA0125A0
:100120004942FFF7DDFFAC4200D04042002C00D036
:10013000494270BDF0B51FB40646002082B00546A6
:100140004024019100901BE0019922460F46304661
:1001500000F020F8049A059B801A994110D31046AC
:100160001946224600F026FA361A8F410197224698
:1001700001200021009F00F01DFA38184D41009029
:100180002046641E0028DFDC019B00982946324689
:1001900007B0F0BD10B5202A04DB0846203AD04055
:1001A000002110BD0B46D340D0402024A21A91401C
:1001B0000843194610BD00000549064A0868504327
:1001C000054A801808604008704701490860704778
:1001D000380000206D4EC64139300000D2B201E037
:1001E0000270401C491EFBD270470022F6E710B592
:1001F00013460A4604461946FFF7F0FF204610BD95
:10020000F0B507460846584087B0C00F0490480034
:100210000E46590040084908BC1A884105D23846A4
:1002200031461E4617460B4602465800400810430A
:100230004CD0300D039040055900400D490D0590FC
:10024000401A0290402872DA18030121000B0905B8
:100250000843019004980092002805D00199524269
:100260000020884100920190029840210A1A0199C9
:10027000009800F09FF905460C466B4607CB00F04E
:10028000A9F9C0197141039A0E0D0023D7175640E2
:100290001A467A40164344D0049A002A2DD0029A76
:1002A000012A039A15DC1205C01A91410126360570
:1002B000001C7141D20F059ED20700930192029655
:1002C0002A46234600F0A6F907B0F0BD384631466D
:1002D000FAE71605224A0F46B218C01AB7410121A3
:1002E0000905001C4F4100187F411146181879413B
:1002F000E20F10436D19644113E0E2076D081543E6
:100300006408C2071443039A01261205C01A9141DA
:100310003605001C7141CE07400830434908C0181B
:1003200051412A46234600F068F9CDE7FFE70498DB
:1003300001224000C117121A00238B410498314654
:10034000C417381AA141EEE730B40124E407634032
:1003500030BC55E730B40124E407614030BC4FE7BE
:100360000000E0FFF0B51FB488B00B990998002495
:1003700048400999C00F490049080991C0070B99E5
:100380000090490049080B9109990898A64608432E
:100390001CD00B990A98084318D0099801244000F2
:1003A000420D4800410D099824050003000B20432D
:1003B00009900B980003000B20430B9050181C4928
:1003C0004018002201901446104605E00020014626
:1003D0000DB0F0BD032801DA034600E003239C467C
:1003E000C11A0AAE0AE05F0008ADED5B4F00F75B93
:1003F0007D430027AA187C41491C5B1E6145F2DD44
:10040000410004AB5A522104120C0A43240C401C34
:100410000828DFDB01980290009970460191009056
:10042000059B049A0799069800F0F4F8D0E70000BD
:100430000DFCFFFFF0B50C465C4085B0E40FE4070F
:1004400003944C000026640859009446490802466B
:100450000296224321D062460A431ED06200570D05
:100460004A000E032303550D012402462C4924059E
:10047000781B1B0B360B4018234326436146009024
:100480001C46501AB44103D30098401C009002E06F
:10049000921800985B41002803DA0020014605B05D
:1004A000F0BD0020012109050746864611E064469B
:1004B0001D46141BB54106D36546521BB341744615
:1004C00007430C43A646CD07400849082843921825
:1004D0005B4105460D43EAD11046184313D06046F0
:1004E000194650407140084306D06046101AB34187
:1004F00006D20122002306E000220123DB0702E0EE
:100500000122D2435310009874460105381C614102
:10051000029C039D0019694100F06FF8BFE70000DD
:10052000FD03000070B54B005B0803430BD04B008C
:100530005C0D002633466542B341D417AD1AA34182
:1005400002DB0020014670BD12053018514170BD1C
:100550000EB505490291002100910A460B46019112
:1005600000F058F803B000BD3304000070B5CD0FA3
:100570004A0009030123090B1B0519430B4BED0727
:100580000024520D9A4201DA002070BD074B34332B
:100590009A4203DC9A1AFFF7FDFD02E00449511864
:1005A00088402C43F1D0404270BD0000FF030000A2
:1005B000CDFBFFFF10B5202A04DB0146203A914015
:1005C000002010BD914020239C1A0346E3401943AC
:1005D000904010BD10B5202A06DBCB170846203A04
:1005E0001041C1170B4306E00B461341D0402024B5
:1005F000A21A91400843194610BD10B5002B08DA25
:100600000024401C614192185B411A4301D140080B
:10061000400010BDF0B51FB482B005460C0003D0F9
:10062000084601F0C8FB02E001F0C5FB203002469D
:10063000009021462846FFF7BDFF049B059A04461B
:100640000F4618431143084314D0184610431BD0DB
:10065000009840210A1A18460599FFF79BFD0546A8
:100660000E46009A05990498FFF7A4FF084305D0A9
:10067000012004E02046394607B0F0BD0020C11734
:1006800005430E432C43374300990E986305401AE7
:100690007905E40A00220C43FD0A0A3002D5002045
:1006A0000146E9E70105101969410C9C0D9D0019EF
:1006B0006941FFF7A2FFDFE70EB5C217C10F504037
:1006C000CA0740180021054B0293019200910A4687
:1006D0000B46FFF79FFF03B000BD0000330400008E
:1006E00010B5002904DB0124E40740428C41214677
:1006F000002B04DB1C460123DB075242A3418B4243
:1007000000D1824210BD0000064C0125064E05E0D6
:10071000E36807CC2B430C3C98471034B442F7D322
:10072000FFF7CAFCB82E0008D82E000870B50446A2
:1007300000688168490720D581681026490700298B
:1007400005DA8168890702D481683143816000F04D
:10075000E3FB05460DE000F0DFFB401B022808D953
:10076000A06B3043A063E06B01210843E0630846BF
:1007700070BD206880684007EDD4002070BDF8B5DA
:100780000446006881688907890F012928D101681A
:10079000C90702D1C168090422D581680522114028
:1007A0001025012601290FD18168022211438160A1
:1007B00021680320086000F0AFFB07460CE000F062
:1007C000ABFBC01B022807D9A06B2843A063E06BDA
:1007D0003043E0630120F8BD20688068C007EED197
:1007E0000020F8BDF8B5044600200090206881681C
:1007F0008907890F012905D10168C9072CD1C16872
:10080000090429D48168154A1026114001250029C0
:1008100015D1816829438160124811490068FFF7AA
:100820005FFC00E0401E00900028FBD100F074FB4C
:1008300007460CE000F070FBC01B022807D9A06B34
:100840003043A063E06B2843E0630120F8BD2068DB
:100850000068C043C007EDD10020F8BD170000803C
:1008600040420F000C00002010B5102000F07CFA70
:1008700010BD0000F8B50025044620340095227D07
:10088000012A39D00122227503689E68760767D451
:10089000384F4E68BE424DD09E6A0F78BA4016431C
:1008A0009E620123C26A1B079A421FD0012A1DD0F3
:1008B000022A1BD0032A19D0042A17D0052A15D0E2
:1008C000062A13D0072A11D002688B68566976076A
:1008D000760FB3420AD05369DB08DB00536100682E
:1008E00042690B7A5B075B0F1A4342610A68102A60
:1008F00004D0112A02D038E00220F8BD1E488368D7
:10090000102A07D00122920513438360086810283B
:1009100003D02AE00122D205F6E7194817490068FA
:10092000FFF7DEFB0A21484300E0401E009000284C
:10093000FBD11AE0986A0E78B24090439862096839
:10094000102901D0112910D10B488268102904D038
:10095000012189058A43826007E00121C905F9E781
:10096000816B2022114381630125002020752846D8
:10097000F8BD0000011000000027014040420F00B8
:100980000C0000200068006C70470000F8B50026DD
:100990000446002805D0A06B25462035002802D04B
:1009A00007E00120F8BD0020E0632875204600F034
:1009B000A9F8A06B1022C006002870DB20688168AF
:1009C00049076CD4A16B1301994302231943A16316
:1009D00081688907890F012905D10168C9070FD1ED
:1009E000C16809040CD4C16818239943A36819434A
:1009F000C160206801696368890089081943016141
:100A00002068C1683D4B1940C160207E617E800333
:100A1000C9030843A17E4B031843A36A012B02D0EC
:100A200001231B0300E000231843E36818432369F4
:100A3000022B09D0002318432B79E57E5B00184375
:100A40000123012D02D00AE00423F4E7002927D076
:100A5000A16B20252943A163E16B1943E163E1699F
:100A60000D46FF3DC23D02D0256A29430843216857
:100A7000CD680543CD600125E16A2D07A94213D059
:100A8000012911D002290FD003290DD004290BD040
:100A9000052909D0062907D0072905D010E028E04C
:100AA000012109040843DAE721684D69ED08ED00EA
:100AB0004D6121684D69A78D7F077F0F3D434D61D3
:100AC0002168C9680E4D2940814207D10020E063AA
:100AD000A06B80088000401CA06308E0A06B02218E
:100AE00088431043A063E06B1843E063012630465F
:100AF000F8BDA06B1043A063F8E700001902FEFFE9
:100B0000E7FF3F8310B586B0044614216846FFF71F
:100B10006CFB0F492068884218D10E488269411544
:100B20000A43826182690A400592426909020A43C6
:100B30004261406908400590032000900190002028
:100B4000029009206946C00600F01AF906B010BDEF
:100B50000024014000100240F8B5044640692546D3
:100B600020350E4608280BD02068C068C00709D081
:100B7000A06B20210843A063002028750120F8BD48
:100B8000082700E00C2700F0C7F9009011E0701C66
:100B90000FD0002E05D000F0BFF90099401AB042E6
:100BA00007D9A06B04210843A06300202875032007
:100BB000F8BD206800683842E9D0A06B01214902E5
:100BC0000843A0632068C16809058A0F0C21002A28
:100BD0001AD1A27E002A17D10268120714D58268A2
:100BE00053070122002B08DB43688B434360A06B53
:100BF000130298431043A06306E0A06B2023184320
:100C0000A063E06B1043E063207E002801D12068E0
:100C100001600020F8BD000070B504462168002086
:100C20008968490721D425462035297D01291CD012
:100C300001212975617E012904D02046FFF7D2FDEC
:100C4000002811D1A16B0A4A1140FF220132114341
:100C5000A1630021E163297522681C2111602168CC
:100C60008A6804231A438A6070BD022070BD0000A8
:100C7000FEF1FFFF70B5054604462035287D0128AA
:100C800007D001262E752046FFF750FD002802D020
:100C90000CE0022070BD2046FFF771FD002805D151
:100CA000A16BFF22013291433143A16300212975D9
:100CB00070BD0000F8B50024254610284FD1FF2153
:100CC000084600F0FDFD0927254EFF0602E0641CE2
:100CD000B44244D81021384600F00AF90028F6D072
:100CE000002403E01E48641C844238D81021384692
:100CF00000F0FEF80128F5D000263446002703E076
:100D00001748761C86422AD809201021C00600F018
:100D1000EFF80028F4D003E011486D1C85421ED87E
:100D200009201021C00600F0E3F80128F4D00D4896
:100D30007200015D4906090E0155AA4202D2012244
:100D40001143015500267F1CFFB23546082FDBD327
:100D5000641CE4B2052CD1D3024901204871F8BDCE
:100D600050C300001C00002010B504494A6902422B
:100D700002D04861FFF79EFF10BD00000004014053
:100D8000FCB500230124A1E027462A469F403A40B3
:100D900073D04D68012D05D0022D03D0112D01D047
:100DA000122D16D185680326AC465D00AE46AE40D6
:100DB0006546B543AC46CE687546AE4065462E43A3
:100DC000866046680D79BE43ED06ED0F9D403543C4
:100DD0004560C6685F000325BD40AE46AE4335465C
:100DE0008E68BE402E43C6604E68022E01D0122E81
:100DF00014D1DE08B60036180196366A5D07B4468F
:100E0000EE0E0F25B54000966646AE43B4460D691A
:100E1000009EB54066462E43019D2E6206687546CB
:100E2000AE430D79AD07AD0FBD40354305604D684C
:100E3000ED004AD5284DAE692643AE61AD699E08E6
:100E4000ED07ED0F0095254DB6007519AC46AD6860
:100E50009E07360F0F27B740BD430927FF06B8424C
:100E600001D1002710E01E4FB84201D101270BE04D
:100E70001C4FB84202D1022706E026E01A4FB842C2
:100E800001D1032700E00527B7402F436546AF6037
:100E9000164E35684F689543FF0300D515433560FE
:100EA00075684F689543BF0300D515437560B568F5
:100EB0004F689543FF0200D51543B560F5684F684C
:100EC0009543BF0200D51543F5605B1C0A681546C3
:100ED000DA4000D058E7FCBD00100240000001409D
:100EE0000004004800080048000C004800040140CD
:100EF0000069084000D001207047426913460B404A
:100F00001B0491430B4383617047002A01D0816128
:100F10007047816270470000014880687047000098
:100F200000000020024881680278891881607047BB
:100F30000000002010B5064801681022114301602E
:100F4000002000F007F800F027F8002010BD000096
:100F50000020024070B504460D4D7D202978C00068
:100F6000FFF7BEF801460B480068FFF7B9F800F03C
:100F700043FB002809D1042C07D200222146401E41
:100F800000F02AF800206C6070BD012070BD0000E8
:100F9000000000200C00002008B5084881690122EB
:100FA00011438161816911400091C26901040A43C2
:100FB000C261C0690840009008BD000000100240F6
:100FC000002805DBC106C90E0120884001490860E0
:100FD0007047000000E100E010B500F01BFF10BDFD
:100FE000F8B505460068354CC00352D5E0690026C7
:100FF000C00007D4E16920040143E161E1690140D7
:10100000012600912E480168C90510D40168821597
:1010100011430160FFF780FF074604E0FFF77CFF04
:10102000C01B642824D826480068C005F6D5206A6D
:1010300003273F02384020D06968394081421CD0E4
:10104000206A226AB843012109040A432262226A03
:101050008A4322622062C0070FD0FFF75DFF009035
:1010600008E0FFF759FF0099411A1648814201D95B
:101070000320F8BD206A8007F3D5206A6968B84369
:1010800008432062002E04D0E1690120000781435B
:10109000E1612878C00705D0206BA968800880002E
:1010A000084320632878800605D5206B10218843EB
:1010B000E968084320630020F8BD000000100240EA
:1010C0000070004088130000F8B50F46060059D0A4
:1010D0003A4D2868C007C00FB84209D228684008B6
:1010E0004000384328602868C007C00FB84249D183
:1010F0003068334C81070CD5400704D56068072160
:101100000902084360606068F0218843B1680843C1
:1011100060603078C00726D0706801280ED0216842
:1011200002280ED0890700292CDA61688908890015
:1011300001436160FFF7F0FE00900DE02168890334
:10114000F1E78901EFE7FFF7E7FE0099411A1D4833
:10115000814201D90320F8BD60680C210840716804
:1011600089008842EFD12868C007C00FB8420BD968
:10117000286840084000384328602868C007C00F2E
:10118000B84201D00120F8BD3078400706D560682C
:10119000072109028843F1680843606000F028F8DD
:1011A0006168094A0906090F515CC840074908608F
:1011B0000020FFF7CFFE0020F8BD00000020024015
:1011C0000010024088130000342E00080C0000209C
:1011D0000448054900684968044A4905490F515CBB
:1011E000C84070470C00002000100240442E000848
:1011F00010B514A30FCB88B06C460FC415A30FCB4A
:101200000FC4184A51680C200B4603401648042BA3
:1012100016D0082B14D18B021B0F6C46E45CD26AEB
:1012200004AB1207120F9A5CC90305D500231946B7
:10123000FEF780FF214601E020460C4900F0D2FD78
:1012400008B010BD02030405060708090A0B0C0DBF
:101250000E0F10100102030405060708090A0B0C03
:101260000D0E0F100010024000127A0000093D0020
:10127000FEB5040070D02078DC4DC0074AD0686805
:101280000007800F012807D068680007800F022838
:1012900009D16868C00306D5286880033AD560681C
:1012A0000028E7D036E06168012914D001208004CD
:1012B000002901D0052914D02A68012109048A4394
:1012C0002A602968814329606068002816D0FFF7EA
:1012D00023FE06460EE02868012109040843286021
:1012E000F2E7296801432960F5E7FFF715FE801B47
:1012F00064286ED828688003F7D50BE0FFF70CFE52
:10130000064604E0FFF708FE801B6428F1D8286831
:101310008003F7D420780126800700283CDA68682B
:101320000007800F07D068680007800F022809D1E6
:101330006868C00306D42868800716D5E0680128CD
:101340000AD112E0E0680028286816D030432860EF
:10135000FFF7E2FD074605E043E1FFF7DDFDC01BB7
:101360000228C6D828688007F7D52868F82188435E
:101370002169C900084328600EE040084000286049
:10138000FFF7CAFD074604E0FFF7C6FDC01B0228B1
:10139000AFD828688007F7D42078000722D5E06905
:1013A0000028686A0ED030436862FFF7B5FD074633
:1013B00004E0FFF7B1FDC01B02289AD8686A8007D5
:1013C000F7D50FE0400840006862FFF7A5FD07462B
:1013D00005E09DE0FFF7A0FDC01B022889D8686AE0
:1013E0008007F7D4207804274007002860DA00201F
:1013F0000190E869C00008D4E969B8060143E961D1
:10140000E969014001200091019079480168C9050E
:1014100011D40168821511430160FFF77DFD009032
:1014200005E0FFF779FD0099401A642870D87048EC
:101430000068C005F5D5A06801280AD0002801D0B1
:10144000052810D0286A400840002862286AB8435E
:1014500001E0286A30432862A068002812D0FFF714
:101460005BFD00900AE0286A38432862F1E7FFF745
:1014700053FD0099411A5F48814249D8286A800784
:10148000F5D50DE0FFF748FD009006E0FFF744FDBD
:101490000099411A574881423AD8286A8007F5D402
:1014A0000198002804D0E969012000078143E9611F
:1014B0002078C00635D5606901280CD0401D686BC6
:1014C00023D038436863686B400840006863FFF7C7
:1014D00023FD064622E0686B38436863686B30433F
:1014E0006863FFF719FD064604E0FFF715FD801B52
:1014F00002285BD8686B8007F7D5686BF8218843B2
:10150000A169C900084368630BE0B8436863F4E766
:101510004CE0FFF701FD801B022847D8686B80076D
:10152000F7D4206A00285ED069680907890F02296C
:1015300042D0012636060228286805D0B04328602C
:10154000FFF7EAFC044633E0B0432860FFF7E4FC11
:10155000074604E0FFF7E0FCC01B022826D82868F5
:101560008001F7D4E86AE16A000900010843E862F3
:10157000616AA06A084369683D22120491430843E6
:101580006860286830432860FFF7C6FC044604E022
:10159000FFF7C2FC001B022808D828688001F7D595
:1015A00021E0FFF7B9FC001B022801D90320FEBD92
:1015B00028688001F5D416E00128F8D06868E96A47
:1015C00001221204636A02409A420AD10907E26AC0
:1015D000090F914205D10F2189040840A16A884270
:1015E00001D00120FEBD0020FEBD00000010024021
:1015F0000070004088130000094910B5401E884261
:1016000001D9012010BD074C60610321081F00F0C3
:1016100001FC0020A06107202061002010BD000017
:10162000FFFFFF0000E000E010B5040003D0A06F52
:10163000002802D007E0012010BD002174200155D0
:10164000204600F027F82420A06720680168490898
:1016500049000160204600F0D1FA0128ECD0606A10
:10166000002802D0204600F031FA206841680122AB
:10167000D2029143416020688168082291438160D1
:1016800020680168012211430160204600F084FABD
:1016900010BD000010B586B0044614216846FEF760
:1016A000A4FD1249206888421ED111488269012197
:1016B00089030A43826182690A4005924269C9002E
:1016C0000A4342614069084005900C2000900220C6
:1016D0000190002002900320039001200490092033
:1016E0006946C006FFF74CFB06B010BD003801404C
:1016F00000100240FEE70000FEB500241349144824
:1017000000940194029412C001250426011D046076
:1017100070C1047444748474C574FF21C23184613F
:101720004161014618310C7105620838FFF72EF946
:10173000280301906946029600940548FFF79AF83D
:10174000694603480095FFF795F8FEBD0024014067
:1017500048000020F0B587B014216846FEF745FD2B
:101760003D484269012189050A43426142690A40B4
:101770000592426949110A43426142690A40059251
:10178000426949000A4342614069344E084005906D
:10179000002203213046FFF7B8FB09200022A021D8
:1017A000C006FFF7B2FB0022E3212D48FFF7ADFB97
:1017B000F1130122C803FFF7A8FB012218212848D2
:1017C000FFF7A3FB0324012502276846B0C0694642
:1017D00030460394FFF7D4FA10200090214801907E
:1017E0000026092069460296C006FFF7C9FAA02024
:1017F0006A460394A1C209206946C006FFF7C0FAF1
:10180000402000900920019669460296C006FFF725
:10181000B7FAE3206A460394A1C269461048FFF76D
:10182000AFFA092000036A46039461C26946C00307
:10183000FFF7A6FA18206A46039461C26946084871
:10184000FFF79EFA002211460720FFF7C5FB07208D
:10185000FFF7B6FB07B0F0BD0010024000140048CF
:10186000000400480000211010B50A480849016032
:101870004B214902416000218160C16001618161A9
:10188000C1610C22016242614162FFF7CDFE10BDD1
:1018900000380140880000207047704710B50020D4
:1018A00000F068FF012109200903C006FFF720FBB3
:1018B000002801D0002010BD012010BD704700009D
:1018C000F8B507460E46012000F054FF0924012117
:1018D000E406002209032046FFF717FB0022082137
:1018E0002748FFF712FB01210022C9032046FFF71A
:1018F0000CFB234C00253846A840000601D50122E8
:1019000000E00022012109200903C006FFF7FDFACB
:10191000012208212046FFF7F8FA0022082120467C
:10192000FFF7F3FA6D1CEDB2082DE4D3002509276B
:10193000FF063046A840000601D5012200E0002243
:10194000012109033846FFF7E0FA01220821204669
:10195000FFF7DBFA002208212046FFF7D6FA6D1CBC
:10196000EDB2082DE5D30122D40321463846FFF716
:10197000CCFA002221463846FFF7C7FAF8BD00002E
:1019800000040048F8B50646012000F0F3FE0925E2
:101990000121ED06002209032846FFF7B6FA0022CE
:1019A00010211948FFF7B1FA01210022C903284686
:1019B000FFF7ABFA2F46144D00243046A040000636
:1019C00001D5012200E00022012109033846FFF77A
:1019D0009CFA012210212846FFF797FA00221021D5
:1019E0002846FFF792FA641CE4B2082CE5D30122E2
:1019F000D40321463846FFF788FA002221463846AC
:101A0000FFF783FAF8BD00000004004810B5FFF7A7
:101A100083FA11498A6890421BD90A328A60087B8E
:101A2000C00717D10A684868904213D0904201DD80
:101A3000401E00E0401C4860C117890F0918890842
:101A40008900401A054940180078C043C0B2FFF72A
:101A500099FF10BD0020FAE7340100204C2E000849
:101A600010B5FFF75FFA10BD70B594B0302168462D
:101A7000FEF7BBFB002401250F9412200595009072
:101A800010200E9410941394049006900D94052049
:101A90001294C0040C94039502260A90119408969F
:101AA00009940B946846FFF7E3FB07200C900E9413
:101AB00001210D960F940CA8FFF706FB10A81095B6
:101AC0001294FFF78DFA14B070BD704710B5818C79
:101AD000C90707D001684A6801235B049A43836AF7
:101AE0001A434A60818C890707D501684A68012337
:101AF0001B049A43C36A1A434A60818C490707D57D
:101B000001684A6801239B049A43036B1A434A60A5
:101B1000818C090707D501684A680123DB039A43D2
:101B2000436B1A434A60818CC90607D502689168E5
:101B300001231B039943836B19439160818C8906B0
:101B400007D501688A6801235B039A43C36B1A4374
:101B50008A60818C490612D503685A6801210905FB
:101B6000046C8A4322435A60026C8A4207D102689D
:101B7000516803235B059943436C19435160818C81
:101B8000090607D501684A680123DB04806C9A4383
:101B900002434A6010BD0000F8B5044600268030BC
:101BA0000660FFF7B9F9054620680068124F000784
:101BB00009D501212B46002249052046009700F057
:101BC000ABF800280DD12068006840070BD5012133
:101BD0002B46002289052046009700F09DF800283A
:101BE00001D00320F8BD2020A067E067266660349E
:101BF00026750020F8BD0000FFFFFF0170B5044608
:101C000080682169E269084361690025114308433E
:101C100021680A683C4B1A4002430A602168486800
:101C2000032212039043E26810434860A169206ACE
:101C3000084321688A680B231B029A4302438A6087
:101C40003248006B8007800F16D0012818D0022878
:101C500018D0032812D010210120E369C0032C4AB8
:101C60002C4E83422BD100290ED002290FD00429FB
:101C70000FD008293FD110E00021EDE70221EBE76A
:101C80000421E9E70821E7E7FFF7A2FA03E010469D
:101C900003E0FFF7ADFA002831D0616840004A0840
:101CA0008018FEF71DFA80B201461039B14222D8E1
:101CB0001849491C01400007400F08431DE0002956
:101CC00006D0022907D0042907D0082913D108E03B
:101CD000FFF77EFA03E0104603E0FFF789FA0028D9
:101CE0000DD061684A081018FEF7FAF980B2014673
:101CF0001039B14201D9012501E02168C8600020F6
:101D00006066A066284670BDF369FFFF00100240C0
:101D100000127A00EFFF0000FFB581B005460F46C4
:101D2000044660350A9E39E0701C37D0FFF7F4F89E
:101D30000499401AB04222D8002E20D020680168B1
:101D400049072BD5C069C043000527D4012021686D
:101D5000C002086220680168FF22A132914301603D
:101D6000206881684908490081602020A067E067F9
:101D70008034206000202875032005B0F0BD206865
:101D80000168FF22A13291430160206881684908FF
:101D9000490081602020A067E067EBE72068C16907
:101DA0003846884305D0002103988142BCD00020EA
:101DB000E3E70121F8E72021020C01D010211046B1
:101DC000020A01D010460839020901D01046091F45
:101DD000820801D01046891E420801D0881E704733
:101DE000081A7047F8B5040C8BB2264682B25E43DF
:101DF0000D0C1046370C58433604801900217941E8
:101E000016466E43370C36048019794126466E43D8
:101E10008919F8BD8307FF22DB0E9A408907090E56
:101E20009940002808DB830809489B001B181868A4
:101E300090430843186070470007000F0838830874
:101E400004489B001B18D86990430843D861704729
:101E500000E400E000ED00E0F8B504464F1EC800C5
:101E60000838211815461E46086849683A46062370
:101E70009A4310D02A463346FEF774FA3A46D20007
:101E8000083AA3181A687F1E5B68FEF7B9F90622A4
:101E90003B469343EED1022F23D0042F11D0062FBF
:101EA0002FD12A463346FEF75DFAE36AA26AFEF7AF
:101EB000A7F92A463346FEF755FA636A226AFEF707
:101EC0009FF92A463346FEF74DFAE369A269FEF709
:101ED00097F92A463346FEF745FA63692269FEF709
:101EE0008FF92A463346FEF73DFAE368A268FEF70B
:101EF00087F92A463346FEF735FA63682268FEF70B
:101F00007FF9F8BD002210B5134610460149FEF7CF
:101F100091FA10BD0000F03F10B50122FEF702FB60
:101F200010BD002210B5134610461146FEF782FA86
:101F300010BD02E008C8121F08C1002AFAD170477C
:101F40007047002001E001C1121F002AFBD1704739
:101F500001490860704700004400002070B5FEF79A
:101F6000F7FA0B22D243FEF7DDFA184E0022334671
:101F7000FEF7F8F904460D4602460B4600203146AE
:101F8000FEF7E2F902460B4620462946FEF752FAD2
:101F90000F4C00222346FEF7E5F900222346FEF708
:101FA00049FA00F06FFC00220A4BFEF743FA0A4A96
:101FB0000A4BFEF725F902460B4600200849FEF7BA
:101FC00039FA084A084BFEF7BFF970BD000014400B
:101FD000006AF84000DCAE4083DBB5DCE1796B3FA2
:101FE0000000F03F666666666612714070B5064690
:101FF00014460D460C2000F0FDFD002809D0068097
:10200000857084800021064A81609168002902D190
:10201000906070BD11468A68002AFBD1886070BD4F
:102020002C00002010B5134CA068002803D02078A5
:10203000002803D00AE00021084616E001202070A5
:10204000FEF76AFFA168898840186060207801283F
:1020500008D1FEF761FF6168884203D90020207033
:1020600000F074FBA0688178008800F0D1FE207831
:1020700010BD00002C00002008B50020FFF782FCF6
:10208000FE48FEF7A2F8FE4D0226287BFF223043D1
:102090002873182001212860F5320846FFF7A6FFB3
:1020A000F84C002201212046FEF72FFFF64F0022B8
:1020B00002213846FEF729FF002201213846FEF7AB
:1020C00024FF092000228021C006FEF71EFF092000
:1020D00000222021C006FEF718FF00220221204620
:1020E000FEF713FF002280213846FEF70EFF002284
:1020F00040213846FEF709FF002220213846FEF72E
:1021000004FFE24CFF202072C02060721920606042
:10211000607CFB2108406074FF209130214614311F
:102120000860297B02200143D84F00262973143F01
:10213000D748FEF771FDD749D548FEF70DFD0028B9
:10214000F9D1D348FEF71EFCB100C9194A68761CC4
:102150008018F6B24860022EEAD3CD48FEF78AFD19
:102160003868401C386032280DD100263E6032218C
:102170007868FDF7B5FF7E60F8603221B868FDF73A
:10218000AFFFBE603861B88980B2FFF7E7FEFEF7A7
:10219000EDF9C14E7060388A80B2FFF7DFFEFEF7BE
:1021A000E5F937460C37B0607879C0074ED000208B
:1021B00078713879302849D13878C10601D540097D
:1021C00000E0FF2020727978B44800F06BFA1030FC
:1021D0002060B978480918D0627CF720024048098D
:1021E000627440016072C806C00FA072607CFB225E
:1021F0001040CA07520F104360740A070AD5FD2128
:10220000084001210843607411E0607C08221043FB
:102210006074E8E7490702D50221084301E0FD2187
:102220000840400840006074FEF776FEE0609B487E
:10223000F9780F3000F036FA401C2074009800281E
:1022400004D1012132220846FFF7D0FE09204021A7
:10225000C006FEF74DFE002805D18F48FB22143042
:102260000179114001718C4F3878C1060FD4E97A99
:10227000C90915D0122108433870012132220846BD
:10228000FFF7B4FE607CFB210840607408E0FD218C
:1022900008403870E97AC90902D1EF210840387046
:1022A000387801070FD4E97A490615D50921084382
:1022B0003870012132220846FFF798FE617CFB202E
:1022C0000140617408E0400840003870E97A49062E
:1022D00002D4F72108403870387881060FD4297B62
:1022E000C90715D02421084338700121322208463D
:1022F000FFF77CFE607CFB210840607408E0FB2156
:1023000008403870297BC90702D1DF2108403870A6
:10231000387881070AD5217AFF2916D0FF2121724A
:10232000617CFD22490849001140617472686A604D
:1023300021682960237A042B67D008DC002B5AD04F
:10234000012B3ED0022B70D16BE00121E7E7062B79
:1023500071D0FF2B69D150484B4E143001790022C7
:1023600049084900017101213046FEF7CEFD0927D9
:10237000FF06002280213846FEF7C7FD00222021FB
:102380003846FEF7C2FD002202213E48FEF7BDFDA1
:10239000002280213046FEF7B8FD00224021304661
:1023A000FEF7B3FD002220213046FEF7AEFD374890
:1023B000002114300173FF2191310160FF2068601A
:1023C00032E0C10702D06168491E61604007606861
:1023D00001D5401C6060C11C2060914202DA00F00F
:1023E0006FF922E0401F904202DD00F023FA1CE06A
:1023F00000F0E0F919E0C20701D0491E2160400752
:10240000EDD52068401C2060E9E7C20701D0491ED5
:102410002160400702D52068401C206000F076F95A
:1024200003E000F0C7F9FF20286020681E280CDDBB
:102430001E200DE0FFE7C20701D0491E21604007C2
:10244000D3D52068401C2060CFE7102801DA102087
:10245000206060681E2801DD1E2002E0102801DADD
:1024600010206060207AFF287DD009200122802181
:10247000C006FEF74AFD607C000711E0D2040000B0
:1024800044010020001400480004004820010020FE
:1024900048000020FFFF000010000020502E000820
:1024A00015D5FDF789FE794E3146FDF72FFE00293F
:1024B00011D0FDF781FE3146FDF728FE002920D01E
:1024C000FDF77AFE3146FDF721FE00292FD0607A14
:1024D000C02802D011E0C02060726D4E0022202181
:1024E0003046FEF712FD002240213046FEF70DFD7A
:1024F000012280213046FEF708FD607A402802D094
:1025000011E040206072624E002220213046FEF72A
:10251000FCFC002280213046FEF7F7FC012240211E
:102520003046FEF7F2FC607A802802D011E080206D
:102530006072574E002240213046FEF7E6FC002232
:1025400080213046FEF7E1FC012220213046FEF7D3
:10255000DCFCA07A012824D04E4901200873002217
:1025600002214D4800E033E0FEF7CFFC607C4107DC
:1025700006D5297BF92211402973FF212960696062
:10258000C0073FD0FEF7C8FC217C404BE2685943AE
:10259000511888422ED9FF202072607C40084000EC
:1025A00027E0012202213C48FEF7AFFC3948002118
:1025B00001730CC808389342D8D1002A02DCFF21ED
:1025C000913103E0FF2391339A42CFDB0160CDE7E5
:1025D000607C800716D5FEF79FFC217C2B4BE268C0
:1025E00059435118884205D901202072607CFD2191
:1025F00008406074FEF790FC800503D5287BFD2120
:1026000008402873254E307941072CD4810711D416
:10261000C10733D002210843307101221C48FEF764
:1026200074FC287B042108432873307941071AD4AD
:10263000800723D53079C10720D1FD2108403071B2
:10264000002202211248FEF760FC287BFB21084093
:1026500028733079042108433071FEF75DFC306047
:10266000307940070AD5FEF757FC0D4A31688918C2
:10267000884203D93179FB200140317100F0F0FA32
:10268000FFF7D0FC0090FFF7C1F94AE560EA0000CF
:1026900000040048340100200014004824000020F9
:1026A00020BF02000909024609010020135C8B4289
:1026B00004D0401CC0B20F28F8D30F207047000090
:1026C00010B5092000222021C006FEF71EFC0022C2
:1026D00001210B48FEF719FC0A4802680A484168C4
:1026E00014308A4203DB01794908490005E0D21C15
:1026F0008A4203DA017901221143017110BD000001
:1027000000040048200100201000002010B509201E
:1027100000222021C006FEF7F8FB00220121094813
:10272000FEF7F3FB084881681430032903DC0179C4
:102730004908490004E0062903DD0179012211431B
:10274000017110BD000400481000002010B5084CB5
:10275000A068002805D08168002903D0A16000F09E
:102760003FF810BD00F03CF80020A06010BD000054
:102770002C00002010B586B0044614216846FDF7F1
:1027800034FD01200003009003200390002001216C
:10279000002C02D0012C03D004E00291019001E052
:1027A0000191029009206946C006FEF7E9FA06B0D9
:1027B00010BD000010B5092000222021C006FEF740
:1027C000A4FB002201210448FEF79FFB0348017986
:1027D00049084900017110BD000400482400002090
:1027E00010B5002823D0124B0022001F196803E007
:1027F000814203D80A4649680029F9D1002A0AD043
:102800001368841A9C4204D100681818106010469E
:1028100002E0506000E01860002907D002680B1A3F
:10282000934203D10B68D21802604968416010BD21
:102830003C00002010B5092001222021C006FEF72F
:1028400064FB0D4802680D480146436814310C488A
:102850009A4205DC0A79520852000A71002207E008
:10286000D21C9A4207DD0A7901231A430A711A46DB
:102870000121FEF74AFB10BD2001002010000020BE
:1028800000040048F0B5C54A00248FB091420ADA2E
:102890004B005B08934206D801254A006D05EA42C9
:1028A00005D1002803D0FFF737FB0FB0F0BD01259D
:1028B0002D05A94219DA034308D0002910DA0120B6
:1028C000FFF746FBFFF72DFB0FB0F0BD0220FFF72F
:1028D0003FFBFFF717FB0122D20751400FB0F0BDBD
:1028E0003524E4433622FDF71DFE0A15AC4B1219C0
:1028F000D4180A03120BAB49AB4B56182E40314685
:10290000594011430192321512190B920022FDF722
:102910001BFD019A0446921C1003A44E000B0D46A9
:102920007E44032860D2204673683268FDF7D8FEE3
:102930001CD10B98002815D0FDF7BEFE04460E46AC
:102940009B4A9C4BFDF70EFD0D4607469A4A9B4B52
:1029500020463146FDF706FD3A462B46FDF750FC72
:102960000FB0F0BD716830680FB0F0BD944A954B60
:1029700020462946FDF7F6FC0022934BFDF7EAFCC2
:1029800006460F4622462B4610461946FDF7EAFC3E
:1029900032463B46FDF7E6FC06460B980F460028FC
:1029A0001DD0FDF789FE824A824B05910490FDF708
:1029B000D9FC32463B46FDF7CDFC22462B46FDF7BF
:1029C000C3FC04460D467C4A7C4B05990498FDF7F0
:1029D000C9FC22462B46FDF7B7FC0FB0F0BD0B46F5
:1029E000324620462946C4E0012300229B072046A8
:1029F000FDF706FC02460B4620462946FDF71AFD68
:102A000006460F460B98FDF757FE32463B460591AA
:102A1000049010461946FDF7A5FC09910C906B49EE
:102A20000198099B421800920C9A19461046FDF72E
:102A300099FC024607910A90654901980B1A65486E
:102A4000019303217844079BFFF706FA079B0A9A34
:102A5000FDF788FC0E905F480D9104217844079B98
:102A60000A9AFFF7F9F9099B0C9AFDF77BFC019B89
:102A7000009A1A4300920D9B0E9AFDF7C1FB009A33
:102A800001910C90002A4DDD0022D24320462946B8
:102A9000FDF748FD22462B46FDF764FC00910A90A5
:102AA0000B9800282BD0424A424B05990498FDF719
:102AB00059FC07910E90019B0C9A00990A98FDF71A
:102AC0009FFB32463B46FDF74DFC079B0E9AFDF7F8
:102AD00097FB009B0A9AFDF73DFC22462B46FDF72B
:102AE00033FC04460D46344A344B05990498FDF7EF
:102AF00039FC22462B46FDF727FC0FB0F0BD019BA9
:102B00000C9A0A98FDF77CFB32463B46FDF72AFCFF
:102B1000009B0A9AFDF71EFC22462B46FDF71AFC85
:102B20000FB0F0BD0B98002827D0214A214B059902
:102B30000498FDF717FC0791009020462946019B59
:102B40000C9AFDF701FC32463B46FDF70BFC079B58
:102B5000009AFDF7F9FB22462B46FDF7F5FB0446EC
:102B60000D46154A154B05990498FDF7FBFB2246C7
:102B70002B46FDF7E9FB0FB0F0BD0B46204629467A
:102B80000C9AFDF7E1FB32463B46FDF7EBFB224694
:102B90002B46FDF7DFFB0FB0F0BD00000000F07F1B
:102BA00001FCFFFF645F09000000F03F8C0500009E
:102BB000763C7935EF39EA3D0000E0FE422EE63FF3
:102BC000555555555555D53F0000E03F86EBF9FF6B
:102BD00051B8060030040000FEF7ACF9FEF744FFE0
:102BE000FEF7B8FDFEF788FDFEF73EFEFFF744FA5C
:102BF000FEE70000F0B50B30C108C900144F0026F5
:102C0000144A0FE003688B420BD38B4205D95C1A40
:102C10004318456830C3083B00E04368136002C0B6
:102C200004E0021D10680028ECD13046002803D1D2
:102C30003868002801D00020F0BD064A0648106020
:102C4000064A121AD208D20044C001203860D7E7E1
:102C5000400000203C0000205C01002058050020BE
:102C600070B5694C694D6068FF2865D00A21FDF791
:102C70004DFA295CF720FEF723FE0A216068FDF774
:102C800045FA695CEF20FEF71BFE2068FF2859D04B
:102C90000A21FDF73BFA295CFB20FEF711FE0A2111
:102CA0002068FDF733FA695CDF20FEF709FE207B20
:102CB000002142078025002A00DA80218007402673
:102CC000002800DA3143FD20FEF7FAFD0021FE2046
:102CD000FEF7F6FDFEF7E2FDE17AC0074908C00FF6
:102CE00049000143E17200217F20FEF7E9FDFEF774
:102CF000D5FDE17AC007FD22800F11400143E1724A
:102D00000021BF20FEF7DCFDFEF7C8FDE17AC00719
:102D1000FB22400F114001430A070020E172002A04
:102D200006DBCA0728D008221143E172090723D520
:102D3000E17ACA070CD013E00021F720FEF7C0FDAE
:102D400000219FE70021FB20FEF7BAFD0021ABE741
:102D5000F7221140BF2220721140E17209070BD502
:102D6000217A491CC9B221721E2905D32072E17A49
:102D7000CA0701D03143E172E17ACA0606D48A0754
:102D80001BD510221143E172C90616D5E17A8A07D4
:102D900007D4EF22114049066072490EE172C9065C
:102DA0000BD5617A491CC9B261721E2905D36072C4
:102DB000E17A8A0701D52943E172E17A8A0606D4CD
:102DC0004A071FD520221143E17289061AD5E17AFC
:102DD0004A0709D4DF221140E172A072227B520817
:102DE0005200227389060DD5A17A491CC9B2A1727D
:102DF0001E2907D3A072E07A400703D5207B01216A
:102E00000843207370BD0000440100206E2E0008AE
:102E100010B5074B002804D001211846FEF76DF8C5
:102E200010BD002201211846FEF76FF810BD00000A
:102E3000001400480000000000000000010203042C
:102E4000060708090000000001020304804020106A
:102E50008040C020A060E0109050D030B070F008EA
:102E6000040C020A060E01098088848C828AFAC04A
:102E70009ED6E4767EC2FEF604FA97999999D93FD8
:102E8000AF788E1DC571CC3F9FC678D0099AC33FDD
:102E9000935555555555E53F599322942449D23FB2
:102EA000DE03CB966446C73F44523EDF12F1C23F79
:102EB0000000000000000000D82E000800000020E4
:102EC00048000000321F0008202F000848000020A2
:102ED000100D0000421F0008010000000400000067
:102EE0000000000000127A00000000000000000056
:102EF00000000000000000000000000000000000D2
:102F000000000000000000000000000000000000C1
:102F100000000000000000000000000000000000B1
:04000005080000B13E
:00000001FF
